:020000040000FA
:1000000001308A00D9290000831A0A28A500030EAE
:10001000A6000F288312A500030EA600A6140A0846
:10002000AD008A018313A50E0408A7002008A800CC
:100030002108A9002208AA002308AB002408AC006C
:1000400083128B1E25280B193A28270884002808BC
:10005000A0002908A1002A08A2002B08A3002C0850
:10006000A4002D088A00260E83008312250EA618F0
:1000700083160900643081000030061C013033050E
:1000800003195428AE0A0319AF0A2F08063C0318B7
:100090005328FF3A031D50282E08CF3C031853283D
:1000A000AF01AE01B00A5828AF01AE01B001B101F5
:1000B0000B118A11252835308400000803196D289A
:1000C0000630A100A001A00B6328A10B62287B30A1
:1000D000A000A00B6928800B60280034B6018F01B6
:1000E0008E0106160F08A3000E08A0000F082302B9
:1000F000031D72282008B7002308B8003808083C00
:10010000031C8828031D87283708663C03187228BB
:100110008F018E0106120F08A3000E08A0000F0821
:100120002302031D8B282008B7002308B8003808D5
:10013000033C031CA128031DA0283708F53C031825
:100140008B288F018E0106160F08A3000E08A00051
:100150000F082302031DA4282008B7002308B800B5
:10016000B808031DB7283708FA3C0318A4280F3035
:10017000B600B61B17298F018E0106125530B80044
:100180005A30B7003608A0000319CB280310B80C6A
:10019000B70CA00BC62837080139B900BA01B90855
:1001A000031DD528BA080319EC280F08A3000E0870
:1001B000A0000F082302031DD5282008B70023083C
:1001C000B8003808033C031CEB28031DEA28370855
:1001D000073C0318D528FF280F08A3000E08A0002D
:1001E0000F082302031DEC282008B7002308B800DD
:1001F000B808031DFF283708FA3C0318EC288F01C4
:100200008E0106160F08A3000E08A0000F08230297
:10021000031D02292008B7002308B800B808031DF1
:1002200015293708FA3C03180229B603B9280F30FC
:10023000B600B61B77298F018E010612F130B80087
:100240004830B7003608A00003192B290310B80C5A
:10025000B70CA00B262937080139B900BA01B90833
:10026000031D3529BA0803194C290F08A3000E08ED
:10027000A0000F082302031D35292008B70023081A
:10028000B8003808033C031C4B29031D4A293708D2
:10029000073C031835295F290F08A3000E08A000AA
:1002A0000F082302031D4C292008B7002308B800BB
:1002B000B808031D5F293708FA3C03184C298F0141
:1002C0008E0106160F08A3000E08A0000F082302D7
:1002D000031D62292008B7002308B800B808031DD1
:1002E00075293708FA3C03186229B60319290F301B
:1002F000B600B61BD7298F018E0106123508B8004B
:100300003408B7003608A00003198B290310B80C75
:10031000B70CA00B862937080139B900BA01B90812
:10032000031D9529BA080319AC290F08A3000E086C
:10033000A0000F082302031D95292008B7002308F9
:10034000B8003808033C031CAB29031DAA29370851
:10035000073C03189529BF290F08A3000E08A00029
:100360000F082302031DAC292008B7002308B8009A
:10037000B808031DBF293708FA3C0318AC298F01C0
:100380008E0106160F08A3000E08A0000F08230216
:10039000031DC2292008B7002308B800B808031DB0
:1003A000D5293708FA3C0318C229B6037929061261
:1003B0004C2A84011F30830583161F149F141F15B8
:1003C0008312AE01AF01B001B101B201B3011A3025
:1003D00083168500293086000108C0390338810062
:1003E000643083128100B53090008F018E018B162E
:1003F000C0308B04850186010030861E0130A000CC
:100400000310200DB5000030051E013035040339FE
:100410000319142A013A0319172A033A03191A2A4D
:10042000013A03191D2A202A0130B200232A0A307A
:10043000B200232A1E30B200232A3C30B200232A05
:100440000A30B200232A8519302A1430B5005B2007
:10045000851D282A04308506B3093230B5005B209B
:10046000331C05113318051585183A2AAF01AE0162
:10047000B001B10130083B3C0318402AB001B10A79
:1004800032083102031C552AB101861D542A6830F6
:10049000B5008B30B4006E280230B400FA30B500DD
:1004A0005B20B40B4E2A452AB30131083202013CCD
:0E04B000031C5C2A05145D2A0510FC2963005C
:02400E00BA3FB7
:00000001FF
